:10000000F32B00308A000408840A820700343F344E
:1000100006345B344F3466346D347D3407347F34BA
:0E0020006F3480348834C034403403340434E8
:10040000013463340534831285013030831685004E
:100410009F01073083129900803083168100080005
:10042000EF308312A0002008831685058312051281
:100430002130A000A00B1A2A0800EF308312A00080
:10044000200883168505831205122130A000A00B19
:10045000272A8316851621308312A000A00B2E2A8E
:100460008316051621308312A000A00B352A080040
:1004700083122008210403193E2A3F2A6E2AA5016F
:10048000A50A4D2A01300310A00DA10DFF3E031D4A
:10049000432A0130A4002408A507A11F502A512A8D
:1004A000422A21082302031D572A20082202031C86
:1004B0005A2A5B2A612A2008A2022108031CA303EE
:1004C000A30201300310A10CA00CFF3E031D622A01
:1004D0000130A502031D6D2A6E2A512A2308A100AE
:1004E0002208A00008008312B201B30103222130C8
:1004F0008312AF00AF0B7A2A00308312A800A90044
:100500003823F32201308312B2070318B30A0030F4
:10051000B30727303302103003193202031C912A2B
:10052000922A942AB201B3013308A9003208A80024
:100530003823003A03199D2A9E2A822A0630831204
:10054000B1001330B000AD30AF00AF0BA52AB00B37
:10055000A52AB10BA52AAC2A812A00288312A5015D
:10056000A601200821040319B62AB72AEE2AA701FA
:10057000A70AC52A01300310A00DA10DFF3E031DDF
:10058000BB2A0130A4002408A707A11FC82AC92A32
:10059000BA2A01300310A50DA60DFF3E031DCA2A7D
:1005A00021082302031DD62A20082202031CD92A6F
:1005B000DA2AE12A2008A2022108031CA303A302CD
:1005C000251401300310A10CA00CFF3E031DE22AEC
:1005D0000130A702031DED2AEE2AC92A2608A10030
:1005E0002508A00008008312A501102240308123B5
:1005F0001D221022C03081238312A7012708343E18
:10060000840083130008013E84000120A600250811
:10061000031D0B2B0C2B1C2B2708343E84000008D9
:10062000031D132B142B1C2B033027020318192B2B
:100630001A2B252BA601252BA501A50A6330270619
:10064000031D232B242B252BA617260881230130DD
:100650008312A4002408A70704302702031C312BAF
:10066000322BFE2A1D2210228D3081231D220800EC
:1006700003308312AD00AE012E08343E8400831394
:1006800080010130AA002A08AE0704302E02031CA4
:100690004A2B4B2B3C2B792BAD1B4F2B502B772B05
:1006A0000A30A0000030A1002908A3002808A200F9
:1006B000382283122108AC002008AB002D08343EFC
:1006C00084002B08831380000A30A0000030A100B2
:1006D0002908A3002808A200AE2283122108A9003D
:1006E0002008A800FF30AA002A08AD07792BA8012E
:1006F000A90128082904031D7E2B7F2B4C2B0130D8
:1007000008008312A200A301DF30A0002008831696
:100710008505831285122130A000A00B8D2B83123A
:10072000221C932B942B972B831605169E2BEF30B0
:10073000A00020088316850583120512213083123C
:10074000A000A00BA12B83122208A0000310200CF4
:10075000A2008316851621308312A000A00BAE2BB9
:1007600001308312A0002008A30708302302031CD5
:10077000BA2BBB2B842BDF30A00020088316850505
:100780008312851283160516831205122130A000EC
:10079000A00BC82B8316851621308312A000A00B56
:1007A000CF2B00308312051A0130A1002108031D50
:1007B000DA2BDB2BE22BEF30A00020088316850517
:1007C000831205122130A000A00BE42BDF3083122E
:1007D000A000200883168505831285122130A00011
:1007E000A00BF02B08000022B8000122B900022261
:0E07F000BA00B401B501B601B7018301732A46
:08400000FF3FFF3FFF3FFF3FC0
:02400E00C431BB
:00000001FF
